S01D000062696E2F6F70656E626C745F73746D3332663736372E7372656389
S31508000000000008204507000895070008950700081E
S3150800001095070008950700089507000800000000E6
S31508000020000000000000000000000000950700081E
S31508000030950700080000000095070008A13400088D
S315080000409507000895070008950700089507000812
S315080000509507000895070008950700089507000802
S3150800006095070008950700089507000895070008F2
S3150800007095070008950700089507000895070008E2
S3150800008095070008950700089507000895070008D2
S3150800009095070008950700089507000895070008C2
S315080000A095070008950700089507000895070008B2
S315080000B095070008950700089507000895070008A2
S315080000C09507000895070008950700089507000892
S315080000D09507000895070008950700089507000882
S315080000E09507000895070008950700089507000872
S315080000F09507000895070008950700089507000862
S315080001009507000895070008950700089507000851
S315080001109507000895070008950700089507000841
S315080001209507000895070008950700089507000831
S315080001309507000895070008950700089507000821
S315080001409507000895070008950700089507000811
S315080001509507000895070008950700089507000801
S3150800016095070008950700089507000895070008F1
S315080001709507000895070008950700080000000085
S3150800018095070008950700089507000895070008D1
S3150800019095070008950700089507000895070008C1
S315080001A095070008950700089507000895070008B1
S315080001B095070008950700089507000895070008A1
S315080001C09507000895070008000000009507000835
S315080001D09507000895070008950700089507000881
S315080001E09507000895070008950700089507000871
S30D080001F09507000895070008B1
S315080001F810B5054C237833B9044B13B10448AFF34B
S3150800020800800123237010BD74040020000000003C
S31508000218BC500008084B10B51BB108490848AFF38D
S3150800022800800848036803B910BD074B002BFBD0AC
S31508000238BDE81040184700BF0000000078040020F9
S31508000248BC500008740400200000000053B94AB9DD
S31508000258002908BF00281CBF4FF0FF314FF0FF30B8
S3150800026800F07EB9ADF1080C6DE904CE00F006F889
S31508000278DDF804E0DDE9022304B070472DE9F0470C
S315080002888C460E460446089D002B50D18A421746CE
S315080002986CD9B2FA82FEBEF1000F0BD0CEF120045B
S315080002A820FA04F401FA0EF644EA060C02FA0EF7E6
S315080002B800FA0EF44FEA1749220CBCFBF9F01FFAAC
S315080002C887F809FB10C642EA064600FB08F3B3425C
S315080002D809D9F61900F1FF3280F02281B34240F2BB
S315080002E81F8102383E44F61AA2B2B6FBF9F309FB97
S315080002F8136642EA064403FB08F8A04509D9E41937
S3150800030803F1FF3280F00A81A04540F20781023BDB
S315080003183C44C8EB040443EA00400021002D62D09F
S3150800032824FA0EF400232C606B60BDE8F0878B4234
S3150800033807D9002D55D0002185E841000846BDE8B3
S31508000348F087B3FA83F1002940F09080B34202D3CC
S31508000358824200F2F880841A66EB03060120B44646
S31508000368002D40D085E81010BDE8F08712B901279E
S31508000378B7FBF2F7B7FA87FEBEF1000F35D1F31BC4
S315080003884FEA17481FFA87FC0121B3FBF8F0220C3D
S3150800039808FB103642EA06460CFB00F3B34207D9B7
S315080003A8F61900F1FF3202D2B34200F2CE801046A7
S315080003B8F61AA2B2B6FBF8F308FB136642EA064435
S315080003C80CFB03FCA44507D9E41903F1FF3202D252
S315080003D8A44500F2B5801346CCEB040443EA004072
S315080003E89CE729462846BDE8F087CEF1200106FA9B
S315080003F80EF307FA0EF720FA01F94FEA1748CE4026
S3150800040849EA0309B6FBF8FA4FEA194408FB1A66DB
S315080004181FFA87FC44EA06430AFB0CF29A4200FADA
S315080004280EF40AD9DB190AF1FF3180F087809A425F
S3150800043840F28480AAF1020A3B449B1A1FFA89F9FA
S31508000448B3FBF8F108FB113349EA034301FB0CF641
S315080004589E4207D9DB1901F1FF326BD29E4269D950
S3150800046802393B449B1B41EA0A418EE7C1F1200E3B
S3150800047822FA0EF48B40234320FA0EF706FA01F403
S315080004884FEA134C26FA0EF63C43B6FBFCF9270C42
S315080004980CFB19661FFA83F847EA064609FB08F7AC
S315080004A8B74202FA01F200FA01FA08D9F61809F170
S315080004B8FF3041D2B7423FD9A9F102091E44F61BBB
S315080004C8A0B2B6FBFCF40CFB146640EA064704FB2C
S315080004D808F8B84507D9FF1804F1FF3028D2B845F7
S315080004E826D9023C1F4444EA0940C8EB0707A0FB83
S315080004F802894F4544464E4614D329D065B3BAEB0C
S31508000508040367EB060707FA0EFECB40CF404EEA10
S31508000518030385E888000021BDE8F0871346F8E656
S315080005281046E0E6B8EB020469EB03060138E5E78E
S315080005380446D8E7114695E78146C0E78A467CE728
S31508000548023B3C4448E708460AE702383E442FE798
S31508000558C245E7D33E46D1E72946BDE8F08700BF3E
S31508000568704700BF70B50F4E0F4D761BB61018BFF3
S31508000578002405D0013455F8043B9847A642F9D11A
S315080005880A4E0B4D761B04F095FDB61018BF0024CD
S3150800059806D0013455F8043B9847A642F9D170BDF0
S315080005A870BD00BFC4510008C4510008CC510008EA
S315080005B8C451000870B4840746D0541E002A41D096
S315080005C8CDB2034602E0621EE4B3144603F8015BA3
S315080005D89A07F8D1032C2ED9CDB245EA05250F2C52
S315080005E845EA054519D903F110022646103E0F2E8D
S315080005F842F8105C42F80C5C42F8085C42F8045C65
S3150800060802F11002F2D8A4F1100222F00F0204F047
S315080006180F041032032C13440DD91E462246043AF9
S31508000628032A46F8045BFAD8221F22F0030204328A
S31508000638134404F003042CB1C9B21C4403F8011B83
S31508000648A342FBD170BC704714460346C2E700BFF5
S31508000658024B13B1024800F005B8704700000000C5
S3150800066879060008002301461A46184600F014B809
S3150800067838B5074D074C2C1BA41005D0013C55F876
S31508000688043D9847002CF9D1BDE8384004F018BD58
S31508000698D0510008CC5100082DE9F047254C2568AB
S315080006A8D5F848410646884692469946C4B36068CE
S315080006B81F2817DC431C76B104EB80050122C5F810
S315080006C888A0D4F8881182401143022EC4F88811EC
S315080006D8C5F808911ED00230636044F820800020CF
S315080006E8BDE8F087144B03B34FF4C870AFF3008026
S315080006F80446D0B1D5F84831002780E88800C5F8FF
S31508000708484138460123C4F88871C4F88C71002E0C
S31508000718E1D0D1E7D4F88C110A43C4F88C21DAE77A
S3150800072805F5A674C5F84841C1E74FF0FF30BDE89E
S31508000738F08700BFD450000800000000DFF834D066
S31508000748002103E00C4B5B58435004310B480C4B13
S3150800075842189A42F6D30B4A02E0002342F8043BB1
S31508000768094B9A42F9D300F0E3FAFFF7FBFE00F0CB
S31508000778DDF8704700000820D05100084000002026
S31508000788740400207404002070420020FEE700006C
S315080007980C4B1968C1F3072353FA81F3C1F30742CF
S315080007A81A440B0E13FA82F39BB2002205E0054998
S315080007B81144087903449BB20132372AF7D95842BB
S315080007C880B270470000002008B5FFF7E1FF044B28
S315080007D89B8F984201D0002008BD012008BD00BFA4
S315080007E80000002008B5064B1A68064B9A4203D142
S315080007F8FFF7EAFF10B908BD002008BD012008BDAB
S3150800080800000020A2E742CE08B5FFF7C1FF014B5A
S31508000818988708BD0000002008B5FFF7E3FF68B908
S31508000828074A084B1A60002304E0064A1A440021BE
S3150800083811710133372BF8D9FFF7E6FF08BD00BF5A
S31508000848A2E742CE0000002038B504460D46FFF759
S31508000858C9FF58B12B1C18BF0123372C08D83BB140
S31508000868044B1C4423792B70012038BD002038BD61
S31508000878002038BD0000002000B595B0254B1A6C3D
S3150800088842F080521A641B6C03F080530093009B55
S31508000898214B1A6842F440421A601B6803F4404325
S315080008A80193019B012307934FF48033089302238E
S315080008B80D934FF480020E9208220F924FF4D872C5
S315080008C810921193129307A800F0E4FC18B1952129
S315080008D8124802F0FBFC00F0FFFF18B19D210F48F3
S315080008E802F0F4FC0F2302930223039300230493D4
S315080008F84FF4A05305934FF480530693072102A893
S3150800090800F02EFF18B1AC21044802F0DFFC15B040
S315080009185DF804FB0038024000700040D850000813
S3150800092808B502F005F8FFF7A7FF08BD30B583B08C
S31508000938002502AC04F8015DFFF7F2FFFFF76CFF2C
S3150800094802F066FC21462846FFF77EFF9DF8073029
S31508000958012B01D102F050FC02F068FCFCE700BF4D
S3150800096870B58EB0394B1A6C42F080521A641A6CFC
S3150800097802F080520192019A5A6C42F480425A64F3
S315080009885A6C02F480420292029A1A6B42F00102E9
S315080009981A631A6B02F001020392039A1A6B42F061
S315080009A802021A631A6B02F002020492049A1A6B7C
S315080009B842F004021A631A6B02F004020592059AB9
S315080009C81A6B42F008021A631A6B02F008020692BA
S315080009D8069A1A6B42F040021A631A6B02F0400232
S315080009E80792079A1A6C42F480221A641B6C03F45D
S315080009F880230893089B8026099601230A930024D6
S31508000A080B940C94124D09A9284600F0A5FF224616
S31508000A183146284601F02CF94FF4005309930A94F5
S31508000A280B9409A90B4800F097FF4FF440730993F4
S31508000A3802230A930B9403230C9307230D9309A9FE
S31508000A48054800F089FF0EB070BD00BF00380240A7
S31508000A580004024000080240000C024010B51E4C73
S31508000A6800228021204601F003F98021204601F062
S31508000A785DF84FF40051194801F058F804F5006478
S31508000A884FF48071204601F051F84FF40071204662
S31508000A9801F04CF8124B1A6C22F480221A641A6B6D
S31508000AA822F040021A631A6B22F008021A631A6BBC
S31508000AB822F004021A631A6B22F002021A631A6BEE
S31508000AC822F001021A631A6C22F080521A645A6CD0
S31508000AD822F480425A6410BD00040240000802400D
S31508000AE8003802400268294B9A424ED1F0B589B0BF
S31508000AF8A3F590431A6B42F000721A631A6B02F058
S31508000B0800720092009A1A6B42F080621A631A6B96
S31508000B1802F080620192019A1A6B42F000621A6327
S31508000B281B6B03F000630293029B3223039302278D
S31508000B38049700260596032506950B24079403A90A
S31508000B48134800F009FF862303930497059606952C
S31508000B58079403A90F4800F0FFFE4FF400530393C8
S31508000B68049705960695079403A90B4800F0F4FE22
S31508000B784FF420530393049705960695079403A9FB
S31508000B88064800F0E9FE09B0F0BD7047008002404B
S31508000B980008024000000240000402400018024013
S31508000BA810B5164B08221A7000225A702721997018
S31508000BB86921D9705B21197145215971104C114960
S31508000BC821600121616022826361A261E2614FF4BA
S31508000BD800032362204601F0CDFC04230A4A0B4988
S31508000BE8204601F009FB0423094A0A49204601F070
S31508000BF83DFB204601F0E6FD10BD00BF900400202D
S31508000C0824230020008002406C230020540A002078
S31508000C18D40A0020A4220020074A1178074B197025
S31508000C285178597091789970D178D9701179197164
S31508000C3852795A71704700BF90040020B009002005
S31508000C48064B1A7802705A7842709A788270DA785F
S31508000C58C2701A7902715B79437170479004002053
S31508000C6838B5124801F0CAFBE8B9104DAC8F2246D0
S31508000C78296C0F4804F013FA2A6B136843F00043EB
S31508000C8813600023AB632B6841F214029A5812F0DA
S31508000C98800F09D0802141F214029950002141F2AF
S31508000CA80802995000E00024204638BD2423002075
S31508000CB8EC3B002038B5194BDC6A02F0E1FB00F181
S31508000CC8FA0505E002F02AFA02F0DAFB854204D3AF
S31508000CD82368002BF6DB012300E0002363B1104BE1
S31508000CE81D880E4CE36A2A460E49986804F0D7F917
S31508000CF82946204601F0F0FA084B1B6841F214020F
S31508000D089A5812F0200F07D0202141F21402995060
S31508000D18002141F20402995038BD00BF242300205F
S31508000D28583B0020EC3B002008B502F0A9FB08BD9B
S31508000D3810B40F4AD2F8883043F47003C2F88830E2
S31508000D480C4B196841F001011960002098601C686D
S31508000D5809492140196009495960196821F480210F
S31508000D681960D8604FF0006393605DF8044B7047CC
S31508000D7800ED00E000380240FFFFF6FE10300024C0
S31508000D8838B5036813F0010F73D10D460446036896
S31508000D983B4A1A404968EB6819432B691943AB69FA
S31508000DA80B4313430360AA68436823F44053134369
S31508000DB843606A69836823F4407313438360314B3D
S31508000DC8984203D1032000F0C9F835E02E4B984223
S31508000DD803D10C2000F0C2F82EE02C4B984203D120
S31508000DE8302000F0BBF827E0294B984204D14FF48D
S31508000DF8406000F0B3F81FE0264B984203D1C020A4
S31508000E0800F078F918E0244B984204D14FF4407062
S31508000E1800F070F910E0214B984204D14FF4405085
S31508000E2800F068F908E01E4B984204D14FF4404098
S31508000E3800F060F900E00020E8B12B68EBB1AA6978
S31508000E48B2F5004F0DD15A0802EB4000B0FBF3F09B
S31508000E584FF6F0730340C0F342001843E0600120E0
S31508000E6838BD00EB5300B0FBF3F080B2E060012018
S31508000E7838BD002038BD002038BD002038BD00BF69
S31508000E88F369FFEF001001400044004000480040A5
S31508000E9800140140004C0040005000400078004013
S31508000EA8007C0040034B9B68C3F30313024AD35CD8
S31508000EB8D840704700380240E0500008034B9B684A
S31508000EC8C3F38223024AD35CD840704700380240ED
S31508000ED8F0500008034B9B68C3F34233024AD35CBD
S31508000EE8D840704700380240F05000080D4B5B6840
S31508000EF803F480030BB90C4B00E00C4B094A506805
S31508000F0800F03F00B3FBF0F05368C3F3881303FB04
S31508000F1800F05368C3F3014301335B00B0FBF3F0F9
S31508000F28704700BF003802400024F40000127A0017
S31508000F3808B5074B9B6803F00C03042B06D0082B4F
S31508000F4801D0044808BDFFF7D1FF08BD024808BD0F
S31508000F58003802400024F40000127A0008B5032875
S31508000F6828D15E4BD3F89030034043EA00405C4BE7
S31508000F78984208D0B0F1031F0DD0013B984212D110
S31508000F88FFF7D6FF08BD554B1B6813F0020F40F054
S31508000F988E80002008BD514B1B6F13F0020F40F0DE
S31508000FA88880002008BDFFF7C3FFFFF77BFFFFF720
S31508000FB891FF08BD0C2826D1484BD3F8903003403A
S31508000FC843EA0040474B984208D0B0F10C1F0CD0B2
S31508000FD8043B984210D1FFF7ABFF08BD3F4B1B688F
S31508000FE813F0020F68D1002008BD3C4B1B6F13F0A5
S31508000FF8020F63D1002008BDFFF79AFFFFF752FFDB
S31508001008FFF75CFF08BDB0F5406F27D1334BD3F81F
S315080010189030034043EA0040334B984209D0B0F178
S315080010280C2F0DD0A3F58063984210D1FFF780FFE7
S3150800103808BD2A4B1B6813F0020F42D1002008BDD1
S31508001048264B1B6F13F0020F3DD1002008BDFFF792
S315080010586FFFFFF727FFFFF73DFF08BD302835D19B
S315080010681E4BD3F89030034043EA00401F4B984282
S3150800107808D0B0F1301F0CD0103B984210D1FFF7BA
S3150800108857FF08BD154B1B6813F0020F20D1002027
S3150800109808BD124B1B6F13F0020F1BD1002008BDA9
S315080010A8FFF746FFFFF7FEFEFFF708FF08BD1048E3
S315080010B808BD4FF4004008BD0D4808BD4FF4004070
S315080010C808BD0B4808BD4FF4004008BD002008BD00
S315080010D8074808BD4FF4004008BD00BF0038024065
S315080010E80200030008000C000008000C200030006D
S315080010F80024F40008B5C02828D1604BD3F89030EE
S31508001108034043EA00405E4B984208D0B0F1C01F3E
S315080011180DD0403B984212D1FFF70AFF08BD574B3E
S315080011281B6813F0020F40F09280002008BD534B4D
S315080011381B6F13F0020F40F08C80002008BDFFF7E4
S31508001148F7FEFFF7AFFEFFF7B9FE08BDB0F5407F1B
S3150800115827D14A4BD3F89030034043EA0040494B1D
S31508001168984209D0B0F1032F0DD0A3F580739842A1
S3150800117810D1FFF7DDFE08BD404B1B6813F0020FC0
S315080011886AD1002008BD3D4B1B6F13F0020F65D1CD
S31508001198002008BDFFF7CCFEFFF784FEFFF78EFE9A
S315080011A808BDB0F5405F27D1344BD3F890300340DB
S315080011B843EA0040344B984209D0B0F1302F0DD09D
S315080011C8A3F58053984210D1FFF7B2FE08BD2B4B02
S315080011D81B6813F0020F44D1002008BD274B1B6F6C
S315080011E813F0020F3FD1002008BDFFF7A1FEFFF755
S315080011F859FEFFF763FE08BDB0F5404F36D11F4BC1
S31508001208D3F89030034043EA0040204B984209D06F
S31508001218B0F1C02F0DD0A3F58043984210D1FFF73F
S3150800122887FE08BD154B1B6813F0020F20D1002056
S3150800123808BD124B1B6F13F0020F1BD1002008BD07
S31508001248FFF776FEFFF72EFEFFF738FE08BD1048B3
S3150800125808BD4FF4004008BD0D4808BD4FF40040CE
S3150800126808BD0B4808BD4FF4004008BD002008BD5E
S31508001278074808BD4FF4004008BD00BF00380240C3
S315080012888000C0000002000300200030008000C073
S315080012980024F400002800F0D78170B582B004460F
S315080012A8036813F0010F65D0A64B9B6803F00C037F
S315080012B8042B0AD0A34B9B6803F00C03082B0DD10B
S315080012C8A04B5B6813F4800F08D09E4B1B6813F479
S315080012D8003F4FD06368002B4CD1B7E16368B3F57C
S315080012E8803F05D1974A136843F48033136020E09A
S315080012F84BB9944B1A6822F480321A601A6822F499
S3150800130880221A6015E0B3F5A02F09D18D4B1A680B
S3150800131842F480221A601A6842F480321A6008E099
S31508001328884B1A6822F480321A601A6822F48022D6
S315080013381A6063687BB102F0ABF8054605E002F06F
S31508001348A7F8401B642800F283817E4B1B6813F4B8
S31508001358003FF4D00EE002F09BF8054605E002F0DF
S3150800136897F8401B642800F27581764B1B6813F4BE
S31508001378003FF4D1236813F0020F54D0714B9B68D1
S3150800138813F00C0F0AD06F4B9B6803F00C03082B5D
S3150800139816D16C4B5B6813F4800F11D1694B1B6827
S315080013A813F0020F03D0E368012B40F05581654A14
S315080013B8136823F0F803216943EAC103136032E08E
S315080013C8E368E3B15F4A136843F00103136002F068
S315080013D85FF8054605E002F05BF8401B022800F2B4
S315080013E83D81584B1B6813F0020FF4D0554A136811
S315080013F823F0F803216943EAC103136013E0514A4D
S31508001408136823F00103136002F042F8054605E065
S3150800141802F03EF8401B022800F22281494B1B685D
S3150800142813F0020FF4D1236813F0080F2AD0636962
S31508001438A3B1444A536F43F00103536702F028F8EF
S31508001448054605E002F024F8401B022800F20A8146
S315080014583C4B5B6F13F0020FF4D013E0394A536F15
S3150800146823F00103536702F013F8054605E002F076
S315080014780FF8401B022800F2F780324B5B6F13F017
S31508001488020FF4D1236813F0040F00F083802D4B64
S315080014981B6C13F0805F0BD12A4B1A6C42F08052F2
S315080014A81A641B6C03F080530193019B012500E025
S315080014B80025254B1B6813F4807F13D1224A13682D
S315080014C843F48073136001F0E3FF064605E001F074
S315080014D8DFFF801B642800F2C9801B4B1B6813F4C6
S315080014E8807FF4D0A368012B05D1164A136F43F001
S315080014F8010313671FE04BB9124B1A6F22F001025A
S315080015081A671A6F22F004021A6714E0052B09D124
S315080015180C4B1A6F42F004021A671A6F42F001025E
S315080015281A6708E0074B1A6F22F001021A671A6F42
S3150800153822F004021A67A368B3B101F0A9FF0646A8
S315080015480CE000BF003802400070004001F0A0FF20
S31508001558801B41F28833984200F28A804C4B1B6FF5
S3150800156813F0020FF2D00FE001F092FF064606E0EC
S3150800157801F08EFF801B41F2883398427AD8444B93
S315080015881B6F13F0020FF3D125B1414A136C23F0F0
S3150800159880531364A369002B6ED03D4A926802F003
S315080015A80C02082A6AD0022B39D1394A136823F063
S315080015B88073136001F06CFF054604E001F068FFCC
S315080015C8401B02285CD8324B1B6813F0007FF5D104
S315080015D8E269236A1343626A43EA8213A26A5208D3
S315080015E8013A43EA0243E26A43EA0263226B43EAA0
S315080015F80273274A5360136843F08073136001F037
S3150800160847FF044604E001F043FF001B022839D8C7
S315080016181F4B1B6813F0007FF5D0002035E01C4AE5
S31508001628136823F08073136001F032FF044604E060
S3150800163801F02EFF001B022826D8154B1B6813F04D
S31508001648007FF5D1002020E00120704701201CE02A
S3150800165803201AE0032018E0012016E0032014E00E
S31508001668032012E0032010E003200EE003200CE01C
S3150800167803200AE0032008E0002006E0012004E031
S31508001688032002E0032000E0032002B070BD00BF7B
S315080016980038024038B52F4B9B6803F00C03042B1F
S315080016A855D0082B01D02C4838BD2A4B5A6802F069
S315080016B83F025B6813F4800F20D0264B5B68C3F3A0
S315080016C88813DC000025690141EAD4616001041B1E
S315080016D861EB0505A90141EA9461A001001B61EBCC
S315080016E80501C01841F100014B0243EAD0534402F0
S315080016F8204619460023FEF7A9FD1FE0154B5B682F
S31508001708C3F38813DC000025690141EAD461600146
S31508001718041B61EB0505A90141EA9461A001001BB8
S3150800172861EB0501C01841F100018B0243EA9053A9
S315080017388402204619460023FEF788FD054B5B6898
S31508001748C3F3014301335B00B0FBF3F038BD03482C
S3150800175838BD00BF003802400024F40000127A00A1
S31508001768002800F09C8070B50446544B1B6803F0AB
S315080017780F038B420BD2514A136823F00F030B430E
S315080017881360136803F00F03994240F08A802368B0
S3150800179813F0020F17D013F0040F04D0484A9368C1
S315080017A843F4E0539360236813F0080F04D0444ABF
S315080017B8936843F4604393604148836823F0F002D2
S315080017C8A368134383600D46236813F0010F2ED0D0
S315080017D86268012A05D13A4B1B6813F4003F0DD1FC
S315080017E861E0022A05D1364B1B6813F0007F05D144
S315080017F85BE0334B1B6813F0020F58D030498B68EF
S3150800180823F0030313438B6001F042FE064606E005
S3150800181801F03EFE801B41F28833984249D8284B8E
S315080018289B6803F00C036268B3EB820FF0D1234B75
S315080018381B6803F00F039D420AD2204A136823F057
S315080018480F032B431360136803F00F039D4232D12D
S31508001858236813F0040F06D019498B6823F4E0525D
S31508001868E36813438B60236813F0080F07D0144AFC
S31508001878936823F46043216943EAC1039360FFF739
S3150800188809FF0F4B9B68C3F303130E4AD35CD84072
S315080018980D4B1860002001F025F8002070BD0120C6
S315080018A87047012070BD012070BD012070BD012060
S315080018B870BD032070BD012070BD00BF003C02400A
S315080018C800380240E050000868040020014B1868F8
S315080018D8704700BF6804002010B582B01C4B1A6C0C
S315080018E842F080521A641B6C03F080530193019BE3
S315080018F8184A136843F48033136001F0C9FD044697
S3150800190805E001F0C5FD001BB0F57A7F1AD8114B22
S315080019185B6813F4803FF4D00E4A136843F4003327
S31508001928136001F0B5FD044605E001F0B1FD001BA2
S31508001938B0F57A7F08D8074B5B6813F4003FF4D0F4
S31508001948002002E0032000E0032002B010BD00BF1B
S315080019580038024000700040F0B583B00024D8E093
S315080019680123A3400A6803EA0205AB4240F0D08087
S315080019784A68122A18BF022A10D1E608083650F80B
S3150800198826C004F0070297000F22BA402CEA020E76
S315080019980A69BA404EEA020240F826200268670039
S315080019A80326BE40F64302EA060E4A6802F0030218
S315080019B8BA404EEA020202604A6802F1FF3E112A5C
S315080019C818BFBEF1010F01D9122A10D1826806EA9A
S315080019D8020ECA68BA404EEA02028260426822EAE1
S315080019E803034A68C2F30012A2401A434260C36856
S315080019F81E408B68BB403343C3604B6813F0805F57
S31508001A0800F08680454B5A6C42F480425A645B6CF7
S31508001A1803F480430193019BA608B21C404B53F874
S31508001A28227004F003039B000F229A4027EA020754
S31508001A383C4A904225D002F58062904223D002F5AE
S31508001A488062904221D002F5806290421FD002F54A
S31508001A58806290421DD002F5806290421BD002F542
S31508001A688062904219D002F58062904217D002F53A
S31508001A788062904215D002F58062904213D10922FD
S31508001A8812E0002210E001220EE002220CE00322F6
S31508001A980AE0042208E0052206E0062204E00722F6
S31508001AA802E0082200E00A2202FA03F33B43023660
S31508001AB81B4A42F826301C4B1A68EB4302EA03060F
S31508001AC84F6817F4803F01D045EA0206164A1660A1
S31508001AD8526803EA02064F6817F4003F01D045EA40
S31508001AE80206114A5660926803EA02064F6817F416
S31508001AF8801F01D045EA02060B4A9660D268134051
S31508001B084E6816F4001F01D045EA0203064AD36058
S31508001B1801340F2C7FF624AF03B0F0BD003802401D
S31508001B280038014000000240003C0140F0B500239F
S31508001B388CE001229A4002EA0104A24240F085801C
S31508001B4806685F000325BD40ED432E4006604FEA50
S31508001B58D30E0EF1080E50F82EC003F00706B6008D
S31508001B680F2707FA06F62CEA060640F82E60866856
S31508001B782E408660466826EA02024260C268154018
S31508001B88C5604FEA930E0EF10205324A52F82550FF
S31508001B9803F00302920097403D402F4EB04225D0ED
S31508001BA806F58066B04223D006F58066B04221D095
S31508001BB806F58066B0421FD006F58066B0421DD08D
S31508001BC806F58066B0421BD006F58066B04219D085
S31508001BD806F58066B04217D006F58066B04215D07D
S31508001BE806F58066B04213D1092612E0002610E0F1
S31508001BF801260EE002260CE003260AE0042608E081
S31508001C08052606E0062604E0072602E0082600E080
S31508001C180A2606FA02F2954217D10E4E0EF102026C
S31508001C2856F8225025EA070746F822700B4D2E6803
S31508001C38E24306EA02042C606C6814406C60AC68DF
S31508001C481440AC60EC682240EA6001330F2B7FF63B
S31508001C5870AFF0BD0038014000000240003C01406A
S31508001C680369194201D0012070470020704700BF58
S31508001C780AB181617047090481617047114A13697D
S31508001C8823F440731361032905D1116948F2040343
S31508001C980B4313610CE0022905D10A4A136943F478
S31508001CA80043136104E0074A136943F00403136108
S31508001CB8044A136943EA002040F480301061BFF3F0
S31508001CC84F8F7047003C024010B431B1012906D045
S31508001CD8022907D14FF4007406E0002404E04FF403
S31508001CE8807401E04FF440740B2800D904300D4B7A
S31508001CF8196921F4407119611A6922431A611A6926
S31508001D0822F0F8021A611A6942EAC00040F0020095
S31508001D1818611A6942F480321A61BFF34F8F5DF869
S31508001D28044B7047003C0240224B1B7D012B3ED0DA
S31508001D3870B50E46044601221E4B1A754CF25030F1
S31508001D4800F0ECF8024668BB4FF0FF3333602368AF
S31508001D58012B0ED16168207CFFF790FF4CF25030BA
S31508001D6800F0DCF8024614490869144B03400B6175
S31508001D7818E0A56811E0217C2846FFF7A5FF4CF274
S31508001D88503000F0CBF80C4A136923F0FA031361B4
S31508001D98024608B1356005E00135E168A3680B44D9
S31508001DA89D42E8D30021034B1975104670BD0220E1
S31508001DB8704700BF3C3B0020003C0240FB7FFFFF0A
S31508001DC810B40A490C6924F440740C610C6944F48B
S31508001DD840740C610C6944F001040C6102604360AC
S31508001DE8BFF34F8F5DF8044B704700BF003C0240B5
S31508001DF8084B1A6922F440721A611A6942F4007289
S31508001E081A611A6942F001021A610160BFF34F8F1D
S31508001E18704700BF003C0240084B1A6922F440721A
S31508001E281A611A6942F480721A611A6942F0010243
S31508001E381A610180BFF34F8F704700BF003C02400C
S31508001E48074B1A6922F440721A611A691A611A69E3
S31508001E5842F001021A610170BFF34F8F704700BF45
S31508001E68003C02401A4BDB6813F0020F04D0194AEB
S31508001E78936943F020039361154BDB6813F0100F41
S31508001E8804D0144A936943F010039361104BDB6836
S31508001E9813F0200F04D00F4A936943F0080393619F
S31508001EA80B4BDB6813F0400F04D00A4A936943F0DA
S31508001EB804039361064BDB6813F0800F04D0054AC8
S31508001EC8936943F002039361F222014BDA60704783
S31508001ED8003C02403C3B0020094B1B69002B0ADAF0
S31508001EE8074B084A5A6002F188325A601B69002B68
S31508001EF803DB00207047002070470120704700BFA9
S31508001F08003C024023016745034A136943F000432E
S31508001F1813610020704700BF003C024038B50446EC
S31508001F280022164B9A6101F0B3FA054608E0B4F1A7
S31508001F38FF3F05D0E4B101F0ABFA401B844219D340
S31508001F480F4BDB6813F4803FF1D10D4BDB6813F0B8
S31508001F58F20F03D0FFF786FF012038BD084BDB6870
S31508001F6813F0010F08D00122054BDA60002038BDAE
S31508001F78032038BD032038BD002038BD3C3B00206F
S31508001F88003C02402DE9F0411E4C247D012C36D038
S31508001F98984617460E46054601221A4B1A754CF2FC
S31508001FA85030FFF7BBFF044618BB032D17D8DFE8E8
S31508001FB805F002070C11F9B23046FFF741FF0EE0AB
S31508001FC8B9B23046FFF728FF09E039463046FFF729
S31508001FD80FFF04E03A4643463046FFF7F1FE4CF257
S31508001FE85030FFF79BFF0446074A136923F001039D
S31508001FF813610022034B1A752046BDE8F0810220BA
S31508002008BDE8F0813C3B0020003C0240507913793A
S3150800201843EA002307480B50D07893781B0443EA11
S315080020280063507843EA002312781343024A8B5018
S31508002038704700BF4080024044800240016841F270
S3150800204818028B5843F400538B507047016841F2C5
S3150800205818028B5843F002038B50704770B59EB030
S31508002068044629B14FF40063C3604FF48043836084
S31508002078E3691BB94FF48063079301E000230793CC
S3150800208820680368354A1A40A168E3681943079B1C
S315080020980B4343F400731343036023681D68012048
S315080020A800F052FC23681D60236840225A602368A2
S315080020B85D68012000F048FC23685D6023680025F8
S315080020C89D602368DD602268936923F0BE031B04BC
S315080020D81B0C43F08003936123689E69012000F076
S315080020E833FC23689E612368DD612368DD69012066
S315080020F800F02AFC2368DD61216841F218054B596E
S31508002108174A1A40174B13434B5123685E59012047
S3150800211800F01AFC23685E51236803F58053124AB7
S315080021281A60236803F580531D68012000F00CFC2B
S31508002138236803F580531D60A369012B06D121681E
S3150800214841F21C028858094B03438B5062690021E7
S315080021582046FFF75BFF1EB070BD00BF0F8120FF4A
S31508002168233FDEF8040020028020C1024000010057
S3150800217810B582B00446002301930268136843F039
S315080021880803136003681B680193012000F0DCFB51
S315080021982368019A1A6002B010BD00BF10B582B054
S315080021A80446002301930268136843F00403136086
S315080021B803681B680193012000F0C6FB2368019A8F
S315080021C81A6002B010BD00BF30B583B005460023BB
S315080021D80193026841F21804135943F48013135102
S315080021E803681B590193012000F0AEFB2B68019A7E
S315080021F81A5103B030BD00BFF0B490F84540012C21
S3150800220830D0012480F84540022480F84440C16251
S31508002218002419E065014F194FF480164E5140F213
S31508002228F45606FB0426BE60C6691EB94E5946F41E
S3150800223840064E515D1EAC4204D2651C01EB45159D
S31508002248FD6000E0F96001349C42E3D3026841F27C
S315080022581003D150012380F84430002380F8453014
S31508002268184600E00220F0BC704700BFF0B490F8AA
S315080022784540012C2DD0012480F84540022480F8D9
S3150800228844408162002416E066018D194FF0004724
S315080022988F5144F2F4566E6040F2F45606FB042653
S315080022A8AE605E1EB44204D2661C01EB4616EE60AA
S315080022B800E0E96001349C42E6D3026841F20C0367
S315080022C8D150012380F84430002380F84530184659
S315080022D800E00220F0BC704790F84530012B00F06A
S315080022E88480012380F84530022380F8443039B9C0
S315080022F8012380F84430002280F8452018467047A4
S31508002308C36A1A68002A07DA122380F844300023B9
S3150800231880F845300120704730B440F2F4529142B3
S315080023280AD9344CA4FB0124A40A40F2F45202FB4D
S31508002338141212B1013400E00124012C3AD11A68AA
S3150800234842F040521A60C36AC1F30C015960C26A66
S31508002358136843F000431360C36ADB68C3622CE062
S31508002368C56A2A6822F040522A6023B9C56A2A68CB
S3150800237842F080522A60C26A40F2F4555560621EDD
S3150800238893420DD1C56A2A6842F000522A601A4A51
S3150800239802FB041202F2F452C56AC2F30C026A601E
S315080023A8C56A2A6842F000422A60C26AD268C262CE
S315080023B8013300E000239C42D2D8036841F2140294
S315080023C89A5812F0040F08D0042141F214029950C1
S315080023D80268002141F20403D150012380F84430F1
S315080023E8002380F84530184601E00220704730BCC3
S315080023F8704700BF0BB002AC0CFAFFFF90F84530E7
S31508002408012B3FD0012380F84530022380F8443059
S31508002418836A1A68002A2DDB1A6812F4807F18D096
S31508002428826B01328263012A00D1036343631A6807
S31508002438C2F30D42043AC263026B92680264DB680F
S315080024488362012380F84430002380F84530184613
S3150800245870471A6812F4007F07D0036300224263A4
S3150800246801228263DB68836204E0826B013282633D
S31508002478DB688362012380F84430002280F845200F
S315080024881846704702207047F8B590F84430DBB212
S31508002498822B33D016460546822380F844300268D4
S315080024A8146904F01C04038ADB029BB21C438901E5
S315080024B801F4F8610C4344F00104146100F0E8FFE4
S315080024C807460FE000F0E4FFC01BB0F5803F07D3CE
S315080024D8012385F84430002385F845300320F8BDE4
S315080024E82B681C6914F0010FECD12B685B699BB249
S315080024F83360012385F844300020F8BD0220F8BD72
S3150800250890F84430DBB2422B32D070B505464223E8
S3150800251880F844300068046904F01C042B8ADB023E
S315080025289BB21C43890101F4F8610C4344F0030487
S3150800253892B242612B681C6100F0AAFF06460FE0BA
S3150800254800F0A6FF801BB0F5803F07D3012385F866
S315080025584430002385F84530032070BD2B681C6974
S3150800256814F0010FECD1012385F84430002070BD22
S315080025780220704770B582B000230193002800F046
S315080025880881044690F8443013F0FF0F04D100235D
S3150800259880F84530FEF7A6FA804B5A6C42F480421A
S315080025A85A645B6C03F480430093009B7C4B5A681F
S315080025B822F400025A605968226A0A435A60236854
S315080025C803F580531A6842F001021A6000F060FFAA
S315080025D805460CE000F05CFF401BB0F5FA7F06D90B
S315080025E8032584F84450002384F84530D2E023684C
S315080025F803F58052126812F0010FEBD11D6925F018
S315080026081C05FFF763F9674B0344674A934202D8E8
S3150800261845F0080516E0654B0344654A934202D817
S3150800262845F00C050EE0634B0344634A934209D907
S31508002638624B0344624A934202D845F0040501E016
S3150800264845F0100523681D614FF400420021204615
S31508002658FFF756FF054638B101212046FFF7FEFC6D
S31508002668012584F8445095E0FF2000F06DF9636869
S31508002678002B6ED000F00CFF064601AA0121204661
S31508002688FFF702FF00F004FF801B41F288339842E7
S315080026980BD901212046FFF7E1FC012384F84430D1
S315080026A8002384F84530032574E0019B13F0040FD2
S315080026B8E3D04FF4805200212046FFF721FF38B1B6
S315080026C801212046FFF7CAFC012584F8445061E039
S315080026D800F0DEFE064601AA01212046FFF7D4FED1
S315080026E800F0D6FE801B41F2883398420BD90121A7
S315080026F82046FFF7B3FC012384F84430002384F806
S315080027084530032546E0019B13F0200FE3D001AAC4
S3150800271810212046FFF7B8FE38B101212046FFF7F9
S315080027289DFC012584F8445034E0019B13F0040FFE
S3150800273803D04FF40062E26001E00022E26013F081
S31508002748020F02D00023A3601BE04FF48043A36066
S3150800275817E0E368C3F3CF02A368C3F34F031A432A
S3150800276800212046FFF7CCFE38B101212046FFF7A5
S3150800277875FC012584F844500CE040F6FF7000F01B
S31508002788E3F800212046FFF769FC012384F8443062
S3150800279800E00125284602B070BD00BF0038024097
S315080027A80038014000D3CEFEBFE1E40040F1E9FD60
S315080027B83F787D0100796CFCFF596202001F0AFA0E
S315080027C87FF0FA0238B590F84530012B1AD004463E
S315080027D8012580F84550022380F84430FFF7C8FCE5
S315080027E82046FFF7DBFC2046FFF7EEFC2046FFF7FE
S315080027F825FC2046FFF72AFC84F84450002084F874
S31508002808450038BD022038BD064AD36823F4E0637C
S315080028181B041B0C000200F4E0601843024B034338
S31508002828D360704700ED00E00000FA0530B4144B99
S31508002838DB68C3F30223C3F10704042C28BF042466
S315080028481D1D062D01D9DD1E00E00025012303FA0A
S3150800285804F4013C2140A940AB40013B1A400A4315
S31508002868002806DA00F00F001201D2B2054B1A54F6
S3150800287803E01201D2B2044B1A5430BC704700BFA9
S3150800288800ED00E014ED00E000E400E00138B0F1E6
S31508002898807F0AD2064B5860F021064A82F8231030
S315080028A80020986007221A6070470120704700BF09
S315080028B810E000E000ED00E010B5094B4FF0FF32DC
S315080028C81A6200241C625A625C621A611C615A61A7
S315080028D85C619A619C61FEF7C1F8204610BD00BF8D
S315080028E80038024010B504460E4B18784FF47A7330
S315080028F8B3FBF0F30C4A1068B0FBF3F0FFF7C6FF1A
S3150800290858B90F2C0BD8002221464FF0FF30FFF795
S315080029188DFF064B1C60002010BD012010BD01204C
S3150800292810BD00BF70040020680400206C04002055
S3150800293808B50320FFF768FF0020FFF7D3FFFEF767
S315080029480FF8002008BD00BF38B5044600F0A0FD02
S315080029580546B4F1FF3F02D0044B1B781C4400F02F
S3150800296897FD401B8442FAD838BD00BF7004002082
S31508002978014B1880704700BF9804002008B500F07E
S315080029887FFD0F4B1B68984218D30E4B1B783BB933
S3150800299801220C4B1A7080210B48FFF769F906E0EB
S315080029A80022084B1A7080210748FFF761F900F0E2
S315080029B867FD064B1B881844014B186008BD00BF05
S315080029C89C04002096040020000402409804002075
S315080029D808B5002280210248FFF74AF908BD00BF5A
S315080029E80004024008B5FFF7F3FF4FF40051044806
S315080029F8FFF736F9012801D1002008BD012008BDD6
S31508002A080008024008B56420FFF7B2FF08BD00BFFA
S31508002A1808B5FFF7B3FF08BD0022014B5A70704787
S31508002A28A0040020034BFE22DA7018710222A3F8CC
S31508002A3844207047A004002010B5054C00232370D5
S31508002A48FFF7EAFFFF23E3700123A4F8443010BD1B
S31508002A58A0040020064BFF22DA7000221A71597862
S31508002A6859719A71DA711A720622A3F844207047C6
S31508002A78A004002008B50020FFF7D4FF08BD00BF52
S31508002A88084BFF22DA70084A9A6400221A715A71AA
S31508002A989A710721D9711A725A729A720822A3F87A
S31508002AA844207047A0040020F8500008044BFF2271
S31508002AB8DA7042689A640122A3F84420704700BF76
S31508002AC8A004002008B53120FFF7ACFF08BD00BFF9
S31508002AD838B5084CFF23E37000252571657100F0A9
S31508002AE86DFBA071E571257265720723A4F8443059
S31508002AF838BD00BFA004002038B5FFF78DFF0E4C7F
S31508002B0801252570FF23E3701023237100236371C1
S31508002B1800F054FBA07100F05DFBE07100F05AFB71
S31508002B28C0F3072020726572A5720823A4F84430FA
S31508002B3800F0B4FC38BD00BFA004002038B505462F
S31508002B48447800F03BFB0138844203DD2220FFF776
S31508002B5869FF38BD084C6A78A16C201D00F0AAFEEA
S31508002B68FF23E3706B78A26C1344A3646B78013374
S31508002B78A4F8443038BD00BFA004002038B5044680
S31508002B88457800F01BFB0138854203DD2220FFF754
S31508002B9849FF38BD6168084DA9646278281D00F0A8
S31508002BA889FEFF23EB706378AA6C1344AB646378D9
S31508002BB80133A5F8443038BDA0040020F8B5054609
S31508002BC81746002406E015F8013B1C44E4B200F059
S31508002BD8A5FA31464E1E0029F5D13C600120F8BDFC
S31508002BE810B5084CFF23E370E21D4168A06CFFF797
S31508002BF8E5FF207100236371A3710823A4F8443004
S31508002C0810BD00BFA004002038B505460D4B9C6CC6
S31508002C1800F0D4FA6A1C411E204600F043FC18B995
S31508002C283120FFF7FFFE38BD064CFF23E37000F09E
S31508002C38C5FA0138A36C1844A0640123A4F84430E3
S31508002C4838BD00BFA004002038B50446457800F012
S31508002C58B5FA0238854203DD2220FFF7E3FE38BDC0
S31508002C680F4BFF22DA700122A3F84420617831B9A4
S31508002C7800F028FC90B93120FFF7D4FE38BDA21C15
S31508002C88074B986C00F00EFC18B93120FFF7CAFEFE
S31508002C9838BD6378024A916C0B44936438BD00BF0B
S31508002CA8A004002008B54168074B986C00F0FEFBA5
S31508002CB818B93120FFF7B6FE08BD034BFF22DA70B4
S31508002CC80122A3F8442008BDA004002008B500F096
S31508002CD8CBFD034BFF22DA700122A3F8442008BD76
S31508002CE8A004002008B589B200F052FA08BD00BF52
S31508002CF8054B00221A709A6483F84320A3F84420E7
S31508002D089A705A70704700BFA0040020024B1878C2
S31508002D1800B10120704700BFA00400200022024B22
S31508002D2883F84320704700BFA004002008B503783D
S31508002D38FF2B02D1FFF7E0FE50E0334A1278012A4A
S31508002D4860D1C93B352B46D8DFE803F03345454201
S31508002D5845453F363C394545454545454545454537
S31508002D6845454545454545454545454545454545FD
S31508002D78454545454545241E1B2145454527452ABC
S31508002D882D30FFF7DBFE29E0FFF7F8FE26E0FFF710
S31508002D988DFE23E0FFF724FF20E0FFF771FE1DE014
S31508002DA8FFF768FE1AE0FFF755FE17E0FFF744FE3F
S31508002DB814E0FFF729FF11E0FFF746FF0EE0FFF7DB
S31508002DC887FE0BE0FFF76EFF08E0FFF77FFF05E0D9
S31508002DD8FFF778FE02E02020FFF724FE0A4B93F857
S31508002DE84330012B02D11020FFF71CFE064BB3F91E
S31508002DF84410002906DD1846012380F843300330BD
S31508002E08FFF770FF08BD00BFA004002010B5FDF746
S31508002E1827FF48B3444A1080444B9C894FF4006006
S31508002E2800F01AFE84420DD1012000F04FFE3E4BF9
S31508002E381B88CBB101F0CEFDFDF73CFF00223A4BCB
S31508002E481A8011E0394B9C8940F6060000F004FE0A
S31508002E58844209D101F04EFD334B1B8823B1FDF797
S31508002E6829FF0022304B1A8000F00AFB304B1B68FA
S31508002E78984232D303F5FA732D4A1360002413E0F7
S31508002E882C4A682303FB04232B4A1360022000F00C
S31508002E981DFE254B1B8833B101F09CFDFDF70AFF83
S31508002EA80022214B1A800134002CE9D0002412E0B4
S31508002EB8224B03EB8413224A1360052000F006FE12
S31508002EC8194B1B8833B101F085FDFDF7F3FE002287
S31508002ED8154B1A800134002CEAD000F0D1FA194BA8
S31508002EE81B68984206D342F210721A44154B1A60A8
S31508002EF801F0CEFC002413E00E4A682303FB0423E2
S31508002F080D4A1360032000F0E1FD074B1B8833B117
S31508002F1801F060FDFDF7CEFE0022034B1A8001344E
S31508002F28002CE9D010BD00BF583B0020EC3B002020
S31508002F38FC040020743B0020703B0020304200202F
S31508002F48683B0020F00400201F4B1B78002B39D162
S31508002F5810B5FDF725FE00F093FA00F5FA701B4B3D
S31508002F68186000F08DFA42F210730344184A136089
S31508002F7800F018FD174A002313805380164A138059
S31508002F885380164A138053804EF6030000F04AFD14
S31508002F98FDF742FE124C2046FDF752FE0621204652
S31508002FA801F000FF01F01CFF00F070F942F20F7300
S31508002FB8984203D842F2107000F062F90122094BD0
S31508002FC81A7010BD704700BF71040020FC04002069
S31508002FD8F0040020E83B0020E43B0020E03B00200A
S31508002FE8F4040020EC04002008B50022034B1A70EC
S31508002FF8034B1B780BB9FFF7A7FF08BD7104002020
S31508003008EC0400200F4B1B78012B19D170B40E4B1A
S315080030181D68EE692E62002306E01A1DC45C2A4460
S3150800302882F8204001339BB28AB29342F5D3043220
S31508003038A5F86420012385F866301E44EE6170BC45
S31508003048704700BFEC040020703B002008B5044B0D
S315080030581B78012B01D1FFF7D9FE002008BD00BF58
S31508003068EC04002010B5274B1C68274B1B7813F077
S31508003078400F09D00123E3610023A4F8643084F8DB
S31508003088663084F8673010BD13F0010F02D00022AD
S3150800309884F8672013F0040F09D094F86730012BD9
S315080030A805D1B4F8641004F1200001F059FB164B59
S315080030B81B7813F0080F10D094F86630012B0CD142
S315080030C8002384F86630B4F8641031B1012384F813
S315080030D8673004F1200001F043FB0B4B1B7813F013
S315080030E8020F0ED0094B19880B1F402B09DC94F8E0
S315080030F8673033B9064B18680439C9B20430FFF784
S3150800310815FE10BD703B0020643B0020583B00208C
S315080031186C3B002008B5FFF775FC08BD08B5FFF736
S3150800312877FC08BD08B5FFF7E3FD00F0F7F80022BD
S31508003138014B1A7008BD00BF7204002000B583B0A1
S315080031480DF107010F4800F01FF9012807D10022E1
S315080031580D4B1A709DF807100A48FFF7E7FD0DF1A1
S3150800316807010848FFF772FF012807D10322064B13
S315080031781A709DF807100348FFF7D8FD03B05DF8E5
S3150800318804FB00BF0005002072040020704700BF3A
S3150800319838B504460D46084B1B7813B9C9B200F072
S315080031A8D7F8054B1B78032B03D1E9B22046FFF75E
S315080031B829FFFFF7B3FD38BD72040020044B1B78BE
S315080031C8013B012B01D9402070470020704700BFFA
S315080031D872040020044B1B78013B012B01D94020BF
S315080031E870470020704700BF7204002008B5FFF733
S315080031F88DFD00B1012008BD08B5FFF7F5FE0322CD
S31508003208024B1A7000F048F808BD00BF7204002087
S3150800321808B500F025FBFFF77DFF00F00FF900F071
S315080032283DF9FFF77FFF00F045F808BD08B5FFF739
S3150800323875FF00F017F9FFF781FF00F001F808BDE0
S3150800324808B5FFF7D3FF012813D00A4B1B78012BC3
S315080032580FD100F015F9084B1A68084B1B68134478
S3150800326803F5FA73984204D30022024B1A7000F049
S31508003278FBFA08BD44050020400500204805002043
S31508003288014B1860704700BF40050020014B1868BD
S31508003298704700BF4005002008B5044B1B78012B72
S315080032A803D100F0EDF8024B186008BD440500206C
S315080032B84805002008B50122034B1A70FFF7ECFFF2
S315080032C8FFF7BEFF08BD00BF4405002008B5FFF795
S315080032D825FFFCE7054BDB6913F0200F04D0034BE9
S315080032E85B6A037001207047002070470048004059
S315080032F810B5094B986200F0C3F800F10A0405E016
S31508003308FFF70CFF00F0BCF8844204D3024BDB69D4
S3150800331813F0800FF4D010BD0048004010B588B0EF
S315080033284FF46143019300230293039304930C22F9
S31508003338059206930793054C01A92046FDF720FD3B
S31508003348236843F00103236008B010BD0048004015
S3150800335870B506460D46402903D981210948FFF765
S31508003368B5FF2846FFF7C4FF002406E0FFF7D6FE98
S31508003378305DFFF7BDFF0134A4B2ABB29C42F5D36A
S3150800338870BD00BF0051000870B5244B1C78ACB955
S315080033982348FFF79FFF01283ED1214B1B78013BA5
S315080033A8DBB23F2B38D800F06BF81E4B18600022AA
S315080033B81D4B1A700122194B1A702DE006460D4648
S315080033C8194B1B78013316481844FFF783FF044640
S315080033D8012813D1144B1A780132D2B21A70104B3D
S315080033E81B789A4215D11149304600F063FA002233
S315080033F80A4B1A700C4B1B782B700DE000F040F83E
S31508003408084B1B686433984205D90024034B1C7083
S3150800341802E0002400E00024204670BD4D05002087
S3150800342854050020500500204C05002055050020AD
S315080034380022014B1A60704710E000E008B5FFF754
S31508003448F7FF054B054A5A6000229A60052119605C
S31508003458034B1A6008BD00BF10E000E0BF4B03002D
S3150800346898050020044B1B6813F4803F03D0034AD1
S31508003478136801331360704710E000E098050020D0
S3150800348808B5FFF7EFFF014B186808BD9805002037
S3150800349808B5FFF7F5FF08BD704700BF08B500F087
S315080034A80BF908BD08B500F013F908BD08B500F012
S315080034B845F908BD08B500F087F908BD08B500F054
S315080034C8CBF908BD08B500F057F9034610B100F066
S315080034D8A3F90346184608BD38B50546002419E079
S315080034E8FFF71CFE04EB440293000C4AD358AB4280
S315080034F80ED804EB44018A0008490A445268134462
S315080035089D4205D204EB440083000B44187A38BD63
S315080035180134E4B20A2CE3D9FF2038BD2851000843
S3150800352808B5C1F3080353B90368994209D040F8A6
S31508003538041B4FF4007200F0BDF9012008BD0020F5
S3150800354808BD012008BD00BF2DE9F0410746FEF772
S31508003558C3FC002413E03E68A30006EB03083B44BB
S315080035685D68FFF7DBFD2A46002341460220FEF781
S3150800357809FD40B956F824309D4206D101347F2CFE
S31508003588E9D9012402E0002400E00024FEF7BCFC87
S315080035982046BDE8F08100BF38B50D460B4B98426A
S315080035A807D004460A4B994205D0FFF7CDFF18B94C
S315080035B808E0084C00E0054C29462046FFF7B0FF0E
S315080035C810B938BD002038BD204638BD9C050020F6
S315080035D800800008A00700202DE9F04106460C46A1
S315080035E817461D46DFF86C8001EA08080368B3F138
S315080035F8FF3F04D14146FFF793FF034630B33368CC
S31508003608984505D041463046FFF7C6FF0646D0B16D
S315080036183368E41A34440434FFF780FD331DE31A8B
S31508003628B3F5007F07D308F500713046FFF7B4FFF6
S31508003638064650B1041D17F8013B04F8013B013D45
S31508003648EAD1012302E0002300E000231846BDE87A
S31508003658F08100BF00FEFFFF70B586B004460D4630
S3150800366800230093884201D8012600E0002614B1F9
S315080036780B2D02D802E0002600E00026C6B100237A
S3150800368801930223059301230493FEF725FC09E019
S31508003698FFF744FD0394694601A8FEF745FB20B9E0
S315080036A80134E4B2AC42F3D900E00026FEF72CFC5C
S315080036B8304606B070BD00BF4FF0FF33024A1360AC
S315080036C8024A1360704700BFA00700209C05002027
S315080036D870B54B1E144C241AA3421FD816460D461D
S315080036E80446FFF7F9FEFF281AD028190138FFF70C
S315080036F8F3FEFF2816D00D4B23400D4A934206D1F8
S315080037082B46324621460B48FFF766FF70BD2B4607
S31508003718324621460848FFF75FFF70BD002070BD96
S31508003728002070BD002070BDFFFF1F0800FEFFFFC8
S31508003738008000089C050020A00700204A1E0D4BA3
S315080037481B1A9A4212D870B50D460446FFF7C4FEEE
S31508003758064628190138FFF7BFFEFF2818BFFF2EAF
S3150800376806D001463046FFF777FF70BD0020704740
S31508003778002070BDFFFF1F08114B1B68B3F1FF3F00
S3150800378818D000B583B00E4B59689A681144DA68A0
S3150800379811441A6911445A6911449A691144DA6933
S315080037A88B185B4202AA42F8043D04210548FFF734
S315080037B88FFF01E00120704703B05DF804FB00BFE6
S315080037C89C050020F88100080D4B1A6804331B680D
S315080037D813440C4A126813440B4A126813440B4ADA
S315080037E811680B44043212681A44094B1B681344BF
S315080037F8084A1268D34201D1012070470020704751
S3150800380800800008088000080C800008108000085E
S3150800381818800008F881000808B50D4B1B68B3F135
S31508003828FF3F04D00A48FFF78FFE034668B1094BE5
S315080038381B68B3F1FF3F05D00648FFF785FE034628
S3150800384810B902E0012300E00123184608BD00BFAD
S315080038589C050020A0070020004870470080000843
S3150800386808B500F037F808BD10B5FFF723FE10B9FC
S31508003878FFF7C2FC10BDFFF7B5F810B9FFF7BCFC97
S3150800388810BDFFF783FCFFF7D3FDFFF715F8FFF721
S3150800389815FE064B0340064A9360FFF70FFE446879
S315080038A800F01AF8A047FFF7A7FC10BD80FFFF1F16
S315080038B800ED00E070B508E0461C4D1C0B78037057
S315080038C8FFF72CFC224630462946531E9CB2002A8E
S315080038D8F2D170BD72B6704762B6704710B4013A35
S315080038E80A440BE00C784B7803EB04239BB2184484
S315080038F880B2834201D9013080B202319142F1D3B4
S3150800390807D10B781B02184480B2834201D90130CB
S3150800391880B25DF8044B704770B4C5780D44EDB2B3
S31508003928134CE57083780E0A3344DBB2A3704278E9
S315080039386270007820709CB2A64206D90132D2B2CB
S315080039480B4C62700AB901302070C9B28D420CDA84
S315080039580133DBB2064A93703BB953780133DBB2BD
S31508003968537013B913780133137070BC704700BFCE
S31508003978603B002010B5094C2368014603F108008E
S31508003988FFF7CAFF2368064A1178197251785972DF
S3150800399891789972D278DA7210BD00BF703B002010
S315080039A8603B002000221A4B1A7006E00021194ACB
S315080039B822F813100133164A1370154B1B78002B7F
S315080039C8F4D00022124B1A7008E06822124902FB4A
S315080039D803120021517601330D4A13700C4B1B78DC
S315080039E8002BF2D04FF480620C4B1A800022084B49
S315080039F81A7007E00A4A02EB831200219180013304
S31508003A08034A1370024B1B78002BF3D0704700BF8C
S31508003A18AE090020DC3B0020743B0020AC090020DE
S31508003A283042002000220A4B1A700BE01946094A50
S31508003A3832F813201AB9074B23F8110070470133D7
S31508003A48034A1370024B1B78002BEFD0704700BF50
S31508003A58AE090020DC3B0020030A43EA002080B2B6
S31508003A68704700BF08B5142205490020FFF736FF3E
S31508003A7810B1FFF7F1FF08BD4FF6FF7008BD00BF8C
S31508003A88FA3B002038B50D4D2C7C6B7C03EB0424DF
S31508003A98143CA4B22044082205F11A0180B2FFF7A3
S31508003AA81DFF224605F12201FFF718FF10B1FFF79F
S31508003AB8D3FF38BD4FF6FF7038BD00BFEC3B00207A
S31508003AC808B50620FFF7DEFF08BD00BF70B5A54B91
S31508003AD81C68042800F07181A34BA44A1360A44A01
S31508003AE81360032810D1637E03F00F03032B40F0FD
S31508003AF8D285238A002B40F0CE8508229D4B1A7062
S31508003B08FFF7B0FA00F08CBC02287BD19A4AD37822
S31508003B180133DBB2D37063B993780133DBB29370A0
S31508003B283BB953780133DBB2537013B913780133B1
S31508003B3813700023914A1380914A1380637E052BDC
S31508003B4818BF072B0AD1A37E0133DBB2A376782BDD
S31508003B5840F0A1850023637600F09DBD002B00F098
S31508003B689A85228A002A41D0A27E511EA176002A69
S31508003B7840F09185E27E082A05D0591EC9B2012966
S31508003B880ED8052A0CD1002363768022794B1A7041
S31508003B98FFF768FA14227B4B83F82F2000F00CBD38
S31508003BA8042A03D803219140C9B200E03021A1763E
S31508003BB80132E27603F00F03013B072B00F26B850F
S31508003BC8DFE813F0740208000D00EA036905EA0342
S31508003BD86905EA0300226B4B83F82F206AE2042260
S31508003BE8644B1A70FFF73EFA00F04FBC03F00F0358
S31508003BF8032B40F0508508225E4B1A70FFF732FAFD
S31508003C0800F00EBC052817D15F4B1B689B88002B54
S31508003C1800F041850023534A13605C4A53490A60F9
S31508003C2853490A60564A1380544A13800822514B4E
S31508003C381A7001F021FAC0E0524B9B7B452B40F0E5
S31508003C482A85504A157C537C03EB05214B4A128872
S31508003C58914200F320858DB2484B1D80494B1B7D48
S31508003C6813F03F0F40F01785464B5B7D002B40F05D
S31508003C781285474B1C880CB95B885BB1414BDB8BBB
S31508003C889C4240F008853F4B1A8C414B5B889A4208
S31508003C9840F00185FFF7E6FE4FF6FF73984240F0BD
S31508003CA8FA84384BDB7D062B00F0B880112B23D01D
S31508003CB8012B40F0F084334B93F82230082B40F060
S31508003CC8EA84304B002283F822209B8C4FF6F67242
S31508003CD8934203D909332B4A938402E00833294AC5
S31508003CE89384284B5A8BDA839A8B1A845C83284ADE
S31508003CF852889A8300F0CBBC1C3D204B1D80254A70
S31508003D08214B1A6026E09A880AB31E49898C8A428A
S31508003D181DD1DA8832B11B49498C8A4202D0B2F5DC
S31508003D288A4F14D11A8812B95988002936D04FF6FD
S31508003D38FF718A4202D1588888422FD01149498B87
S31508003D488A4204D10F4A918B5A88914226D0403329
S31508003D580D4A13600C4B1B680F4A9342D3D300F0E5
S31508003D689ABC00BF703B0020223C00206C3B002018
S31508003D785C3B0020643B0020A8090020583B002033
S31508003D882E420020EC3B0020683B0020163C002011
S31508003D98E83B002030420020704200200023AC4A4D
S31508003DA813600221AB4A1170AB4AAC490A60AC49A8
S31508003DB80A60AC4A138001F05FF9AA4B1A88002AF0
S31508003DC800F0698402F11C0189B2A74B1980A74B38
S31508003DD8080A18745974A6490968087A9875112042
S31508003DE8D875083292B2100A40EA0222DA8400220A
S31508003DF883F8282083F829208A885A84CA889A84C6
S31508003E089C4A1088588352889A830A88DA834A888B
S31508003E181A843633914A136000F024BCFFF750FE23
S31508003E284FF6FF73984240F03684934C17E0617E4C
S31508003E38A1B18E4B9A8CA3889A420FD18B4B5A8C78
S31508003E48E3889A420AD1894B5A8B23889A4205D124
S31508003E58864B9A8B63889A4200F046816834864B6B
S31508003E689C42E4D9814B93F82F3003F03F03022B89
S31508003E7814D17E4B9B8C99B2804A13800022804BC2
S31508003E881A7007E07F4A32F8132091425BD0013353
S31508003E987B4A13707A4B1B78002BF3D0734B93F835
S31508003EA82F3013F0040F40F0F683704B142283F872
S31508003EB82F2028216C4A1180502283F82E2093F847
S31508003EC8290093F82D2083F8292093F8281093F8C9
S31508003ED82C2083F8282083F82C1093F8272093F8A9
S31508003EE82B4083F8274083F82B2093F82640644D07
S31508003EF82C7093F82A5083F8265083F82A40013004
S31508003F08C0B283F82D0068B94B1CDBB2574981F853
S31508003F182C303BB9531CDBB281F82B3013B901346A
S31508003F2881F82A40514B5A8C54490A80998C5984ED
S31508003F389A845A8BDA839A8B1A844E4A118859833B
S31508003F4852889A8379E300244D4B1C701CE0194665
S31508003F586822494802FB0302527E1AB9682404FB00
S31508003F68010415E0072A0CD13CB16822424902FB34
S31508003F780312917EA27E914203D93F4A682404FB24
S31508003F88032401333E4A13703D4B1B78002BDED0C1
S31508003F98002C00F080832E4B1C600323A37623761F
S31508003FA80023A3750422E275E376304DAB8CA38013
S31508003FB86B8CE3806B8B2380AB8B638001206076E8
S31508003FC8314B1A7822735A7862739A78A273DB7817
S31508003FD8E373208295F82930E37295F82830A3729E
S31508003FE895F82730637295F826302372FFF7C2FCD6
S31508003FF895F82E0000F0F003502B57DD0022204BD1
S315080040081A704BE003F13602184DAA5C002A4DD007
S31508004018012A03D101331A4A13703FE0022A35D11F
S3150800402803F13702114DAA5C042A2FD101F138038E
S31508004038EA5C39316B5C43EA0222104B1A8040F27B
S315080040480A63934228BF13466382A3822EE000BF01
S31508004058703B0020643B0020163C00206C3B002087
S315080040685C3B00202E420020583B0020EC3B0020F9
S31508004078683B0020E83B0020743B0020A409002088
S31508004088AE090020DC3B0020A809002003F137020E
S31508004098A6498A5C52B11344A54A1370A44B1B78E7
S315080040A819460209053AB3EB820FABDB10229F4B80
S315080040B883F82F209D4B93F82F2042F0020283F8AD
S315080040C82F20022283F83620042283F83720062276
S315080040D883F838200A2283F839202C21954A11803A
S315080040E8602283F82E206EE2934B1C600022934BC5
S315080040F81A708E4B93F82F2012F0040F07D000235E
S31508004108637620228D4B1A70FEF7ACFFC3E2874B05
S3150800411893F82E301B099B0085480370EB1A143B4D
S315080041289BB28448038001F00F01022903D102F0EB
S315080041383F0112290FD013B912F0030F0BD07B4B8E
S31508004148D98C2389994240F03382784B198D638933
S31508004158994240F02D8212F0100F47D0218A002983
S3150800416844D004F10C00FFF7D7FB704B93F82A30BC
S31508004178734A1078834239D16C4B93F82B305178AF
S315080041888B4233D1694B93F82C30927893422DD1D0
S31508004198664B93F82D506A4BDB789D4226D12073DF
S315080041A86173A273E373E37ECBB9237EA27E9B1A5F
S315080041B8DBB2A17DA3EBD103DBB25AB21944C9B26B
S315080041C8A175002A01DA5B425AB2E37DA2EB930293
S315080041D853FA82F2D3B2E37503EBD10323760122AD
S315080041E8564B1A70237EA37600232382617E01F03C
S315080041F80F03013B072B00F24E82DFE813F0080095
S315080042082300A7007301A301BF01D90165014B4B20
S315080042181B7813F0010F00F03E82032363764022D1
S31508004228464B1A7000232382424B188820B1422233
S31508004238424B1A70FFF79EFB0022424B1A80FEF784
S3150800424811FFEDE03D4B1B7813F0010F63D0374B98
S3150800425893F82F3003F03F03122B5CD1334B93F8B6
S315080042682E0000F0F003502B37DD0022304B1A7071
S315080042782BE003F136022D4DAA5C72B3012A03D14D
S3150800428801332B4A137020E0022A16D103F13702AC
S31508004298264DAA5C042A10D101F13803EA5C3931A3
S315080042A86B5C43EA0222284B1A8040F20A6393425F
S315080042B828BF13466382A3820FE003F137021B491E
S315080042C88A5C52B113441A4A1370194B1B7819465B
S315080042D80209053AB3EB820FCBDB03236376134B4C
S315080042E893F82620227293F82720627293F82820DA
S315080042F8A27293F82930E3720120FFF73BFB4222AA
S315080043080E4B1A70002323820A4A13800D4A13801B
S31508004318FEF7A8FE84E02022084B1A70FEF7A2FED4
S31508004328054B1B6800225A76B8E500BFEC3B00200F
S31508004338AE090020583B0020703B0020643B002053
S31508004348603B00202E420020A4090020914B93F8D8
S315080043582F3013F0010F24D011F0100F21D1238A22
S31508004368002B40F098818C4D2888013080B2FFF7E1
S3150800437801FB8A4A137843F0100313702A881AB186
S3150800438843F00203854A1370FEF76CFE0123238265
S31508004398082363760023E37611227E4B83F82F20C1
S315080043A80AE113F0200F10D07A4890F834301A0230
S315080043B890F8353043EA0200794D2E683044286073
S315080043C8754813430288D31A0380734B188848B173
S315080043D811F0100F06D1714A137843F002031370CF
S315080043E8FFF7C8FA6B4A92F8301092F8313003EBA7
S315080043F801239BB26B4A1380A28A934200D80BB951
S31508004408684B1A80674B1B886382644B1B7813F0CA
S31508004418030F00F040810022634B1A80FEF722FE44
S315080044285E4B1B7813F0200F08D000235E4A1380D2
S3150800443863761422574B83F82F20BDE013F0100F2C
S315080044480CD00023584A138001222282042262765D
S31508004458E37611224F4B83F82F20ADE0524A128893
S315080044688AB113F0010F01D000232382238A43B9A6
S31508004478638A9A4201D94C4A13804B4B1B8823827C
S3150800448801E0494A13800023E376484B1A68444BEF
S315080044981A60454B1B884BB1238A3BB128333E4AE1
S315080044A8138018223B4B83F82F2088E03B4B1B7858
S315080044B813F0020F00F0EF802822374B1A801022DB
S315080044C8344B83F82F207AE0344B1B7813F0010F0E
S315080044D800F0E180002363761022304B1A70FEF74D
S315080044E8C1FDD8E02C4B188808B1FFF743FA294BC9
S315080044F893F82F3013F0010F15D0284B1B7813F0BB
S31508004508010F05D0072363760023A376238201E0EB
S31508004518062363760120FFF72DFA10221F4B1A701F
S31508004528FEF7A0FD44E01D4B1B7813F0010F04D0DD
S315080045380523637600232382ADE0174B1B88002BDF
S3150800454836D1A8E0144B188808B1FFF713FA114BAF
S3150800455893F82F3013F0010F0CD007236376002346
S31508004568A3760120FFF706FA10220C4B1A70FEF7FD
S3150800457879FD1DE0084B1B88D3B98CE0074B1B78DF
S3150800458813F0010F00F08780072363760023A376CC
S3150800459881E000BFEC3B0020583B0020643B00202C
S315080045A86C3B0020A40900202E4200205C3B00201A
S315080045B810223C4B83F82F2028223B4B1A80502286
S315080045C8384B83F82E20227A364B83F82A20627ACB
S315080045D883F82B20A27A83F82C20E27A83F82D20F8
S315080045E8227B83F82620627B83F82720A27B83F820
S315080045F82820E27B83F829200622DA75A2885A84BD
S31508004608E2889A84294A1188598352889A83228883
S31508004618DA8362881A84637E13F0100F06D0214B5A
S31508004628002283F8312083F8302006E01D4B062245
S3150800463883F830200A2283F831201A4C4023A375C0
S31508004648194B1B881A0A22746374002384F83530B8
S3150800465884F8343084F8323084F83330FFF730FA87
S31508004668C04360860F4C4523A3730022E273627524
S3150800467822750F490B8801339BB20B80190AA1745E
S31508004688E37422766276FFF7EDF9C04320830022A9
S31508004698084B1A7070BD0023034A1380054A137025
S315080046A870BD00BFEC3B0020583B0020E83B0020CB
S315080046B8A6090020643B0020F8B505460E46254A9B
S315080046C8138801339BB21380B3F5FA4F03D34FF41B
S315080046D88052204B1A8000221F4B1A700CE01F4B81
S315080046E803EB84139F881B4B1888FFF7B5F9874295
S315080046F8E5D00134184B1C70174B1C78002CEED0EB
S3150800470800221A700BE0154A02EB831292881AB92E
S31508004718124800EB831007E001330F4A13700E4B5B
S315080047281B78002BEFD0002088B10A4B1A88130A89
S3150800473843EA02238380C68015B90023036003E091
S315080047482B8803806B88438040230372F8BD0020BA
S31508004758F8BD00BFAC090020AE0900203042002091
S3150800476800290CDD08B58AB2054B1A80054B1B686B
S31508004778834203D00146184600F091FC08BD7047ED
S315080047882E4200205C3B0020F0B400223B4B1A70F6
S315080047983B4E1EE03A4D5A001A4494002E192C5BDB
S315080047A8A4B103EB4305AA00354D2A4452886AB1D9
S315080047B80588AC420AD14488A24207D10C687460BD
S315080047C8898831812F4A1278B27254E001332B4A0C
S315080047D813702A4B1B78072BDCD90022274B1A7033
S315080047E80FE0274D5A001A4494002E192A5B2AB955
S315080047F803EB4304A2002A44528832B101331F4A04
S3150800480813701E4B1B78072BEBD9082B28D10023CE
S315080048181D4A13701D4A1370184A137013E0194A73
S31508004828147803EB4305AA00154D2A44927AA61A6A
S31508004838154D2D78AE4203DD134A1670134A1370C8
S3150800484801330E4A13700D4B1B78072BE7D90F4B0C
S315080048581B780A4A137003EB43039A00084E16445A
S315080048680268334643F8042B0A6872608A889A8075
S31508004878044B1B78B372F0BC704700BFB60900201A
S31508004888B8090020190A0020B7090020180A0020CC
S3150800489810B4154B1C780134E4B21C700022134B73
S315080048A81A7019E012485A001A4491004218415AD7
S315080048B852880A430DD003EB43018A000244927AD0
S315080048C8A21A772A05DD03EB43018A000020084966
S315080048D888500133054A1370044B1B78072BE1D916
S315080048E85DF8044B704700BF190A0020B609002076
S315080048F8B809002010B5324B1B88292B03D800228B
S315080049082F4B1A8010BD00222D4B1A802D4B9B8ADF
S31508004918B3F5807F03D0B3F5007F3FD010BD294B90
S31508004928DA8C294B1B889A4249D1264B1A8D264B75
S315080049385B889A4243D1254C2146A01DFFF724FFE0
S31508004948002204F8022C022204F8012C2168C4F873
S315080049580A10A188E1811E49086820608988A18013
S3150800496844F8100C24F80C1CD4F80A1044F8161C41
S31508004978E28924F8122CE288228222896282124A63
S315080049881188E18052882281082204F80A2C062216
S3150800499804F8092C2A220A4B1A8010BD094BDA8C0E
S315080049A8094B1B889A420AD1064B1A8D064B5B8817
S315080049B89A4204D1054801460630FFF7E5FE10BDC0
S315080049C8583B0020EC3B0020E83B0020023C002036
S315080049D8B009002030B44C4BD98B8AB24FF6FF7316
S315080049E89A420CD1484B188C4FF6FF73984206D159
S315080049F8454B464A1068186092889A8073E0444B7B
S31508004A081B88444800885340184209D13E4B1A8CE3
S31508004A1894B23F4B5B883F4840886340184206D0AB
S31508004A283D4B3E4A1188198052885A8002E03A4B13
S31508004A3819805A8000223A4B1A703A4D16E03948BE
S31508004A485A001A4491004518334A1488425A94421F
S31508004A5809D1314A508803EB43018A0031490A448F
S31508004A685288904206D001332D4A13702C4B1B7876
S31508004A78072BE4D9082B30D1234B4FF0FF321A60A5
S31508004A889A8000221A629A8427490868C3F8060099
S31508004A9889885981C3F8160059831F490888D88414
S31508004AA8498819851A49088898834988D9831A75B7
S31508004AB8012159759A73D973082119745A740622EB
S31508004AC89A740422DA74197306225A733633174A03
S31508004AD813602A22164B1A8014E00B4B55F8042F3C
S31508004AE81A60AA889A80084B0F4A1168C3F80610F4
S31508004AF892885A8108221A7300225A730C4A138814
S31508004B080E33138030BC7047EC3B0020AC510008CC
S31508004B18E83B0020E43B00201C0A0020E03B00207C
S31508004B28B6090020B8090020B00900206C3B00200F
S31508004B38583B002010B504464160FCF7F5F820609C
S31508004B4810BD00BF10B50446FCF7EEF82368C01A76
S31508004B5863689842B4BF0020012010BD352303704E
S31508004B680123437081700330704700BF034636221D
S31508004B78027004224270034A1068C3F80200981D9E
S31508004B88704700BF3C0A002037230370032343708D
S31508004B9801228270C370062303710530704700BF6F
S31508004BA8FF23037001307047074B828C1A80C28C2A
S31508004BB85A80064B028D1A80428D5A80044B028E03
S31508004BC81A80428E5A807047E83B0020E43B002052
S31508004BD8E03B002003463222027004224270034A50
S31508004BE81068C3F80200981D704700BF440A0020E1
S31508004BF810B40346014400242EE01A78332A24D038
S31508004C0806D8032A10D0062A13D0012A21D106E08D
S31508004C18362A15D0FF2A21D0352A1AD10EE0D3F81C
S31508004C280200104A906214E0D3F802000D4A106395
S31508004C380FE0D3F802000B4AD0620AE09C7808E035
S31508004C48D3F80200074AD06103E0D3F80200054A00
S31508004C5810625A78023213448B42CED320465DF846
S31508004C68044B7047200A0020F8B504460123037050
S31508004C784370194B9A6982700025C570174A1068DF
S31508004C886060258180276781154A1268E260256178
S31508004C986561A5619E693246596904F11C0000F0F0
S31508004CA8FEF906F118002044C6F110022946043018
S31508004CB8FBF780FC4022294604F12C00FBF77AFC16
S31508004CC83A46294604F16C00FBF774FC054B18684C
S31508004CD8C4F8EC00F8BD00BF200A0020B45100084B
S31508004CE8E83B0020B851000838B50A4C256828461C
S31508004CF8FFF7BAFF012105F1F000FFF72FFFFFF7CD
S31508004D0843FFFFF74DFF2368C11A1846FFF728FD2A
S31508004D1838BD00BF6C3B002038B50B4C25682846C3
S31508004D28FFF7A2FF032105F1F000FFF717FFFFF7CA
S31508004D381DFFFFF74FFFFFF733FF2368C11A184611
S31508004D48FFF70EFD38BD00BF6C3B002010B5114BB0
S31508004D581C682378022B17D104220F49A01800F0E3
S31508004D688FF998B90D4B9A69596904F11C0000F036
S31508004D7887F968B92069094B5862094B198804F1FB
S31508004D88F000FFF735FF10BD002010BD002010BD4C
S31508004D98002010BD6C3B0020B4510008200A0020F2
S31508004DA8583B002010B582B00C4C6061A161002305
S31508004DB8A3704FF6FF73ADF80430ADF806304FF41C
S31508004DC8864101A8FFF778FC606010B14FF4884364
S31508004DD883800022014B1A8002B010BD200A0020E9
S31508004DE8024B00221A805A80704700BFE83B002011
S31508004DF838B59E4B1B88B3F5937F7FD010D840F201
S31508004E080F12934234D0B3F5887F01D2EBB118E17B
S31508004E18B3F5887F34D040F22512934266D010E164
S31508004E28B3F5AB7F00F0BF8005D840F25512934220
S31508004E3800F0B28005E1B3F5B57F00F0CE8040F208
S31508004E486B12934200F0D080FBE0884B01229A70DF
S31508004E584FF47A721A61FFF747FF844C216904F107
S31508004E680800FFF767FE40F20F132380002300E0CF
S31508004E780123002B00F0EA804FF488727B4B1A80D6
S31508004E887B4B1B7813F0020F05D17A48FFF75AFEB9
S31508004E98002800F0DD80764B1B7813F0020F07D048
S31508004EA8FFF754FF022803D10222704B9A700CE0D0
S31508004EB86E4B1B694EF65F22934202DC5B006B4A17
S31508004EC813616A4B9B78022BC5D14FF47A72674BEC
S31508004ED81A61FFF721FF654C216904F10800FFF7FD
S31508004EE829FE40F225132380002300E00123002B26
S31508004EF800F0B0804FF493725C4B1A805C4B1B78B9
S31508004F0813F0020F05D15B48FFF71CFE002800F0D6
S31508004F18A380574B1B7813F0020F07D0FFF716FF2D
S31508004F28052803D10322514B9A7011E04F4B1B6990
S31508004F3842F21072934207DC4C4A03F57A731361FE
S31508004F489378032BC5D103E00020484B188038BD59
S31508004F584648FFF729FE454D288CFEF77DFD0404D3
S31508004F68688CFEF779FD204340084FF47A7303FBF3
S31508004F7800F0002801DB286103E06FF000423B4B94
S31508004F881A613A4C216904F10800FFF7D3FD40F28B
S31508004F9855132380002300E00123002B5ED04FF42D
S31508004FA8AB72324B1A803348FFF7CCFD002857D02E
S31508004FB82E4B02229A704FF47A721A61FFF710FF85
S31508004FC8FFF7AAFE294C216904F10800FFF7B2FD8C
S31508004FD84FF4B5732380002300E00123002B41D04A
S31508004FE840F26B12214B1A80214B1B7813F0020FE3
S31508004FF804D12048FFF7A6FD002835D01C4B1B789E
S3150800500813F0020F07D0FFF7A1FE052803D10322E4
S31508005018164B9A7011E0154B1B6942F210729342AF
S3150800502807DC124A03F57A7313619378032BC7D101
S3150800503803E000200D4B188038BD0C48FFF7B4FD77
S3150800504889E70022094B1A80022038BD032038BD9B
S31508005058002038BD032038BD002038BD032038BDE0
S31508005068002038BD032038BD002038BD200A00209E
S31508005078643B0020280A002008B5FFF7B9FE08BDDA
S3150800508810B501390244904207D010F8013B11F8CF
S31508005098014FA342F7D0181B10BD002010BD10B54C
S315080050A8431E0A44914204D011F8014B03F8014FF4
S315080050B8F8E710BDF8B500BFF8BC08BC9E467047AF
S311080050C8F8B500BFF8BC08BC9E4670474F
S315080050D4400000206D61696E2E6300000000000028
S315080050E40000000001020304060708090000000086
S315080050F4010203044F70656E424C54002E2E2F2E67
S315080051042E2F2E2E2F536F757263652F41524D43E2
S315080051144D375F53544D333246372F756172742EAB
S315080051246300000000800008008000000100000001
S315080051340000010800800000020000000080010849
S3150800514400800000030000000000020800000200BE
S315080051540400000000000408000004000500000024
S3150800516400000808000004000600000000000C08FF
S3150800517400000400070000000000100800000400F6
S3150800518408000000000014080000040009000000DC
S3150800519400001808000004000A00000000001C08AB
S315080051A4000004000B000000FFFFFFFFFFFF0000E4
S30D080051B4ADDE1223638253638A
S30D080051BCC8B0FF7F01000000E6
S30D080051C4590600081D02000847
S309080051CCF9010008CF
S315080051D0000000002C03002094030020FC0300209C
S315080051E000000000000000000000000000000000B1
S315080051F000000000000000000000000000000000A1
S315080052000000000000000000000000000000000090
S315080052100000000000000000000000000000000080
S315080052200000000000000000000000000000000070
S315080052300000000000000000000000000000000060
S315080052400000000000000000000000000000000050
S315080052500000000000000000000000000000000040
S315080052600000000000000000000000000000000030
S31508005270000000000000000001000000000000001F
S315080052800E33CDAB34126DE6ECDE05000B000000E4
S315080052900000000000000000000000000000000000
S315080052A000000000000000000000000000000000F0
S315080052B000000000000000000000000000000000E0
S315080052C000000000000000000000000000000000D0
S315080055F000000000000000000024F4001000000075
S309080056000101040092
S70508000745A6
